:1000000000308A00E5290000831A0A28A500030EA3
:10001000A6000F288312A500030EA600A6140A0846
:10002000AD008A01A50E0408A7002008A800210839
:10003000A9002208AA002308AB002408AC00831200
:100040008C308400001E26280C1A49288C3084002D
:10005000801E2C288C1A75288C308400801C322835
:100060008C1880298B1E36280B19732927088400C9
:100070002808A0002908A1002A08A2002B08A30034
:100080002C08A400260E83008312250EA6188316C2
:100090000900C608031D512883160C12831206108E
:1000A0005D28460B5628C60199015D283B3045075F
:1000B000840000089900C50AC6030C128A1136286C
:1000C0005F3084000008031974280130A100A001EA
:1000D000A00B6828A10B67284A30A000A00B6E284F
:1000E00000000000800B6528003418080639003A2B
:1000F000031980282E10181218161A08C800702923
:100100002E188D281A08023C031D8C280512D701D1
:100110000430D800D9012E147029483057078400C4
:100120001A0880004830570784000008D907D70A0A
:10013000570B9D280D30D800702958085702031C12
:10014000702901305702483E84000008033C03191F
:10015000AB282E1070290330D902590FB028B228CD
:100160002E10702983168C1283128B1748087F3942
:10017000203C031DBD28C908031D6B29DE015E0854
:10018000073C031CEE2803305E07483E840000084D
:100190001E3C031CD12832305E0784001F308000D3
:1001A000EC2803305E07483E840000085E3C0318DC
:1001B000DF2832305E0784005E308000EC28323069
:1001C0005E07DF0003305E07483E84000008E10060
:1001D0005F08840061088000DE0ABF284A080339EE
:1001E000C7004A081039103C031DF8280510F928EB
:1001F00005144A082039203C031D002985100129D7
:1002000085140608CF39DE004A08C039A000C03086
:100210002002031917298030200203191A294030BF
:10022000200203191C29A00803191E291E29303099
:10023000DE041F29DE161F295E161F291F295E08EE
:10024000860048088039803C031D6B295530BB006F
:100250000230BC002030BD00BE013108BF0020309C
:100260003107FF3AC0000330C1005530C2004708D3
:10027000A000013047020319492902302002031966
:100280004D290330200203195129A00803195529CB
:1002900055290130DF00602056290230DF00602040
:1002A00056290430DF006020562956290830DF0027
:1002B0005F080A3C03185D296B29C60803196129E8
:1002C0006B2906140130C5005F08C6003B08990081
:1002D00083160C1683122E10051683168C168312A5
:1002E0008C128A113628AF08031D7929B00803192A
:1002F0007D292F080319B003AF030B118A1136288B
:100300003A08A000A00803198A290830200203191E
:1003100092299A2910309500DB30831692008312BF
:10032000BA0AA329BB3095003908831692008312BC
:10033000BA01A32901303A02323E84000008831634
:1003400092008312BA0A8C108A113628BA013A0830
:10035000073C031CB22932303A0784003E3080004B
:10036000BA0AA729BA01DB3083169200BB30831288
:1003700095000F3097008316861106308312920085
:10038000910183168C148312FF29D701C6012E1008
:100390000C30831699002430980090308312980016
:1003A00083168C168312002A5C0DAF005D0DB00021
:1003B000AF0DB00DFC30AF05AF08031DE229B0084A
:1003C0000319E4296400DC29003484011F3083050B
:1003D00007309F0064008F3083168100073083123E
:1003E0009F00E030831685001330831285000230B1
:1003F0008316860083128601B001AF01A629C529A4
:10040000E0308B00DD010A30DC00D421DA01640029
:10041000DA08031D0D2A103085065A08F93E031824
:100420005F2A073E6B2A05123F30860505082039F2
:10043000003A031D1D2A31141E2A31105F2A0617A7
:1004400005082039003A031D272AB114282AB110C3
:100450005F2A0613861705082039003A031D322A41
:100460003115332A31115F2A061705082039003A61
:10047000031D3C2AB1153D2AB1115F2A05163F30F4
:10048000860505082039003A031D482A3116492AF5
:1004900031125F2A061705082039003A031D522A37
:1004A000B116532AB1125F2A0613861705082039A0
:1004B000003A031D5D2A31175E2A31135F2ADA0ADA
:1004C0005A08063C0318652ADA01DD016430DC00B5
:1004D000D421072A63000A108A140A118207132AFA
:0C04E0001F2A292A342A3E2A4A2A542ABC
:02400E00453F2C
:00000001FF
